:020000020000FC
:020000000BC033
:10001600C6C002E207B900EE0AB90BB90FEF04B980
:1000260005B90FE1009389000FE30093880009E00A
:100036000093810002E000936F00A8950091600094
:100046000861009360000DE00093600000E6702EEA
:1000560000EA802E00EC902E00247727789404B7CF
:1000660003FD0CC017D003D0FDCF02D001D000D0C5
:10007600A8950AEF202E2220F1F70895A895419819
:10008600459A44EA5EE760EBEDCF4198459A48E928
:100096005EE760EB7C7F419A309BFECF07D0922FC4
:1000A60005D0822F419871FDF0CF29C0332721E07A
:1000B60011D0220F1AD03099239520FD3395309B0D
:1000C600FECFB8F712D03099339530FD7260309B71
:1000D600FECF089506BC12E03099FECF15BD309BC9
:1000E600FECF05BC16B517BD0895A99A06BC12E049
:1000F6003099FECF15BDA99BFECF05BC089591FD95
:10010600019692FD02960027182F292F880F991F16
:10011600810F921F880F991F081B190B2040145F2F
:10012600214022F47160209511952F4F0FEF039512
:10013600185E2340E0F7602E0AE00A951C592F4FFF
:10014600E0F3502E0FEF03951A50E8F7165F402E96
:10015600312E70FD11C0662051F4552019F44598D2
:100166004FEF11C04598052D15D044910CC0459A06
:10017600342C452C4FEC07C04EE74598552019F016
:10018600459A342C452C042D05D05491032D02D0CC
:1001960064910895E8ECF1E0E00FF01D08951FB6B4
:1001A6002A945D9904C07BB845B91FBE18955F991E
:1001B60004C08BB855B91FBE18959BB865B91FBE4C
:0C01C600189581CF9286CCA4A08F808475
:00000001FF
